:020000000150AD
:02000B0021F4DE
:10005000C20075B0FF7590FF75816F758912754B81
:1000600000754C00754D00754E00C201C202C203FE
:10007000C204C206C205C20775453275466475479B
:10008000197548C8754AFA758C38C28ED28CD2A9B7
:10009000D2AF75410175442075430D754220800033
:1000A00020000F30B0057548C8C204200402215E4C
:1000B000D200E54DC4454EFAE54BC4454CF9B909AB
:1000C00005BA0002D207B90905BA0102C207B90987
:1000D00005BA3002D207B90905BA3102C207B90917
:1000E00005BA3202D207B90905BA3302C207B90903
:1000F00005BA5702D207B91005BA0002C207A20713
:10010000B392B3200110B9100D754021854049D23A
:1001100003754F01D201200615B911127548C8C2E6
:100120000475400A854049D203754F01D206300656
:1001300018B96006D205C2AF015030B0057548C885
:10014000C204300404C2AF015200316920010431FD
:100150009701A020060431A401A031D701A0754267
:100160001F75432075442001A030022AC202054EAB
:10017000E54EB40A21754E00054DE54DB4061775E0
:100180004D00054CE54CB40A0D754C00054BE54B94
:10019000B40A03754B0022E54C4410F542854D43EB
:1001A000854E442230032FC203D54F03754F0A7486
:1001B0000AC3954F2323FF90028C93F5420FEF93D0
:1001C000F5430FEF93F5440FEF93F5502540FFC330
:1001D000940340028F4022854B43854C44300313E7
:1001E000C203D54F03754F087408C3954F9002B4EE
:1001F00093F54222C0E0C0D0C082C083300016D543
:100200004513754532D54905854049D203D5460584
:10021000754664D202D54743754705D54805854ADA
:1002200048B204900264D54103754103759000D231
:10023000B5D2B4D2B7E541B40109E54493F590C213
:10024000B58018B40209E54393F590C2B4800CB4AC
:100250000309E54293F590C2B78000D083D082D0E5
:10026000D0D0E032FA9079D993CBEB98FBDB85C400
:1002700064250000FE947DDD97CFEF9CFFDF844472
:1002800024050004000A0818C04060222120200034
:1002900022222000202222002020230020200100F2
:1002A00020202400202525002525200026202000B0
:0C02B000272020FF0A1A0B1B0C1C0D1D40
